:10000000000000308A006A283220A011230803195A
:10001000A0150830A2002E0E1B202E081B202D0E2E
:100020001B202D081B202C0E1B202C081B202B0E08
:100030001B202B081B280F39F63E0318073E0A3EEB
:10004000A400A2030319A011230803192A282202DD
:10005000031831282408031DA011A0193128303EAF
:1000600046280800AE1F0800AB09AC09AD09AE096F
:10007000AB0A0319AC0A0319AD0A0319AE0A2D30F5
:1000800046280C1E4128990003146628211941288E
:100090000800A701A600FF30A607031CA707031C42
:1000A00066280330A500E63057204B28A501FC3E0A
:1000B000A400A509031C6228FF300000A407031850
:1000C0005D28A4070000A50F5C2808008313831295
:1000D00003130800830183164030990020309800F4
:1000E000831290309800A001073083169F00AE3035
:1000F0008312B2004730B1004930B0008030AF0009
:100100000130A700F4308A014A200430A100A30185
:100110003208AE003108AD003008AC002F08AB004B
:100120008A0105200D308A0141208A0180288A0138
:0201300097280E
:02400E00723D01
:00000001FF
